
Z:\tmp\HelloWorld\Build\.elf:     file format elf32-avr

Sections:
Idx Name          Size      VMA       LMA       File off  Algn
  0 .data         00000042  00800100  000009a0  00000a34  2**0
                  CONTENTS, ALLOC, LOAD, DATA
  1 .text         000009a0  00000000  00000000  00000094  2**1
                  CONTENTS, ALLOC, LOAD, READONLY, CODE
  2 .bss          0000019a  00800142  00800142  00000a76  2**0
                  ALLOC
  3 .comment      00000030  00000000  00000000  00000a76  2**0
                  CONTENTS, READONLY
  4 .note.gnu.avr.deviceinfo 0000003c  00000000  00000000  00000aa8  2**2
                  CONTENTS, READONLY
  5 .debug_aranges 00000178  00000000  00000000  00000ae4  2**0
                  CONTENTS, READONLY, DEBUGGING
  6 .debug_info   00001fdb  00000000  00000000  00000c5c  2**0
                  CONTENTS, READONLY, DEBUGGING
  7 .debug_abbrev 00000ab5  00000000  00000000  00002c37  2**0
                  CONTENTS, READONLY, DEBUGGING
  8 .debug_line   00000b0c  00000000  00000000  000036ec  2**0
                  CONTENTS, READONLY, DEBUGGING
  9 .debug_frame  00000618  00000000  00000000  000041f8  2**2
                  CONTENTS, READONLY, DEBUGGING
 10 .debug_str    00000da4  00000000  00000000  00004810  2**0
                  CONTENTS, READONLY, DEBUGGING
 11 .debug_loc    000016c8  00000000  00000000  000055b4  2**0
                  CONTENTS, READONLY, DEBUGGING
 12 .debug_ranges 00000170  00000000  00000000  00006c7c  2**0
                  CONTENTS, READONLY, DEBUGGING

Disassembly of section .text:

00000000 <__vectors>:
   0:	0c 94 34 00 	jmp	0x68	; 0x68 <__ctors_end>
   4:	0c 94 2a 03 	jmp	0x654	; 0x654 <__vector_1>
   8:	0c 94 53 03 	jmp	0x6a6	; 0x6a6 <__vector_2>
   c:	0c 94 51 00 	jmp	0xa2	; 0xa2 <__bad_interrupt>
  10:	0c 94 51 00 	jmp	0xa2	; 0xa2 <__bad_interrupt>
  14:	0c 94 51 00 	jmp	0xa2	; 0xa2 <__bad_interrupt>
  18:	0c 94 51 00 	jmp	0xa2	; 0xa2 <__bad_interrupt>
  1c:	0c 94 ce 03 	jmp	0x79c	; 0x79c <__vector_7>
  20:	0c 94 f7 03 	jmp	0x7ee	; 0x7ee <__vector_8>
  24:	0c 94 51 00 	jmp	0xa2	; 0xa2 <__bad_interrupt>
  28:	0c 94 51 00 	jmp	0xa2	; 0xa2 <__bad_interrupt>
  2c:	0c 94 51 00 	jmp	0xa2	; 0xa2 <__bad_interrupt>
  30:	0c 94 51 00 	jmp	0xa2	; 0xa2 <__bad_interrupt>
  34:	0c 94 20 04 	jmp	0x840	; 0x840 <__vector_13>
  38:	0c 94 7c 03 	jmp	0x6f8	; 0x6f8 <__vector_14>
  3c:	0c 94 a5 03 	jmp	0x74a	; 0x74a <__vector_15>
  40:	0c 94 51 00 	jmp	0xa2	; 0xa2 <__bad_interrupt>
  44:	0c 94 51 00 	jmp	0xa2	; 0xa2 <__bad_interrupt>
  48:	0c 94 fb 02 	jmp	0x5f6	; 0x5f6 <__vector_18>
  4c:	0c 94 cc 02 	jmp	0x598	; 0x598 <__vector_19>
  50:	0c 94 51 00 	jmp	0xa2	; 0xa2 <__bad_interrupt>
  54:	0c 94 51 00 	jmp	0xa2	; 0xa2 <__bad_interrupt>
  58:	0c 94 51 00 	jmp	0xa2	; 0xa2 <__bad_interrupt>
  5c:	0c 94 51 00 	jmp	0xa2	; 0xa2 <__bad_interrupt>
  60:	0c 94 51 00 	jmp	0xa2	; 0xa2 <__bad_interrupt>
  64:	0c 94 51 00 	jmp	0xa2	; 0xa2 <__bad_interrupt>

00000068 <__ctors_end>:
  68:	11 24       	eor	r1, r1
  6a:	1f be       	out	0x3f, r1	; 63
  6c:	cf ef       	ldi	r28, 0xFF	; 255
  6e:	d8 e0       	ldi	r29, 0x08	; 8
  70:	de bf       	out	0x3e, r29	; 62
  72:	cd bf       	out	0x3d, r28	; 61

00000074 <__do_copy_data>:
  74:	11 e0       	ldi	r17, 0x01	; 1
  76:	a0 e0       	ldi	r26, 0x00	; 0
  78:	b1 e0       	ldi	r27, 0x01	; 1
  7a:	e0 ea       	ldi	r30, 0xA0	; 160
  7c:	f9 e0       	ldi	r31, 0x09	; 9
  7e:	02 c0       	rjmp	.+4      	; 0x84 <__do_copy_data+0x10>
  80:	05 90       	lpm	r0, Z+
  82:	0d 92       	st	X+, r0
  84:	a2 34       	cpi	r26, 0x42	; 66
  86:	b1 07       	cpc	r27, r17
  88:	d9 f7       	brne	.-10     	; 0x80 <__do_copy_data+0xc>

0000008a <__do_clear_bss>:
  8a:	22 e0       	ldi	r18, 0x02	; 2
  8c:	a2 e4       	ldi	r26, 0x42	; 66
  8e:	b1 e0       	ldi	r27, 0x01	; 1
  90:	01 c0       	rjmp	.+2      	; 0x94 <.do_clear_bss_start>

00000092 <.do_clear_bss_loop>:
  92:	1d 92       	st	X+, r1

00000094 <.do_clear_bss_start>:
  94:	ac 3d       	cpi	r26, 0xDC	; 220
  96:	b2 07       	cpc	r27, r18
  98:	e1 f7       	brne	.-8      	; 0x92 <.do_clear_bss_loop>
  9a:	0e 94 70 00 	call	0xe0	; 0xe0 <main>
  9e:	0c 94 ce 04 	jmp	0x99c	; 0x99c <_exit>

000000a2 <__bad_interrupt>:
  a2:	0c 94 00 00 	jmp	0	; 0x0 <__vectors>

000000a6 <HeartBeat>:
    // both variables will stay around the next time the function is called
    static uint8_t illuminosity = 0;
    static uint8_t control = 0;
	
    // checks if the direction needs to be changesd
   if (illuminosity >= 255)
  a6:	80 91 43 01 	lds	r24, 0x0143	; 0x800143 <illuminosity.1999>
  aa:	8f 3f       	cpi	r24, 0xFF	; 255
  ac:	19 f4       	brne	.+6      	; 0xb4 <HeartBeat+0xe>
        control = 0;
  ae:	10 92 42 01 	sts	0x0142, r1	; 0x800142 <__data_end>
  b2:	0a c0       	rjmp	.+20     	; 0xc8 <HeartBeat+0x22>
    else if (illuminosity <= 0)
  b4:	81 11       	cpse	r24, r1
  b6:	04 c0       	rjmp	.+8      	; 0xc0 <HeartBeat+0x1a>
        control = 1;
  b8:	91 e0       	ldi	r25, 0x01	; 1
  ba:	90 93 42 01 	sts	0x0142, r25	; 0x800142 <__data_end>
  be:	08 c0       	rjmp	.+16     	; 0xd0 <HeartBeat+0x2a>

    // increases or decreases the brightness, depending on that value
    if (control == 0) 
  c0:	90 91 42 01 	lds	r25, 0x0142	; 0x800142 <__data_end>
  c4:	91 11       	cpse	r25, r1
  c6:	04 c0       	rjmp	.+8      	; 0xd0 <HeartBeat+0x2a>
        illuminosity--;
  c8:	81 50       	subi	r24, 0x01	; 1
  ca:	80 93 43 01 	sts	0x0143, r24	; 0x800143 <illuminosity.1999>
  ce:	03 c0       	rjmp	.+6      	; 0xd6 <HeartBeat+0x30>
    else 
        illuminosity++;
  d0:	8f 5f       	subi	r24, 0xFF	; 255
  d2:	80 93 43 01 	sts	0x0143, r24	; 0x800143 <illuminosity.1999>

    // apply value
    Tcnt2.OCRA = illuminosity;
  d6:	80 91 43 01 	lds	r24, 0x0143	; 0x800143 <illuminosity.1999>
  da:	80 93 b3 00 	sts	0x00B3, r24	; 0x8000b3 <__TEXT_REGION_LENGTH__+0x7e00b3>
  de:	08 95       	ret

000000e0 <main>:
}

int main(void) {
	Usart_Init(250000);
  e0:	60 e9       	ldi	r22, 0x90	; 144
  e2:	70 ed       	ldi	r23, 0xD0	; 208
  e4:	83 e0       	ldi	r24, 0x03	; 3
  e6:	90 e0       	ldi	r25, 0x00	; 0
  e8:	0e 94 d5 00 	call	0x1aa	; 0x1aa <Usart_Init>

    // set configs
    PortB.DDR |= 0x8;
  ec:	23 9a       	sbi	0x04, 3	; 4
    PortB.PORT = 0;
  ee:	15 b8       	out	0x05, r1	; 5
    Tcnt2.TCCRB = 0x5;
  f0:	e0 eb       	ldi	r30, 0xB0	; 176
  f2:	f0 e0       	ldi	r31, 0x00	; 0
  f4:	85 e0       	ldi	r24, 0x05	; 5
  f6:	81 83       	std	Z+1, r24	; 0x01
    Tcnt2.TCCRA = 0x81;
  f8:	81 e8       	ldi	r24, 0x81	; 129
  fa:	80 83       	st	Z, r24

    // start timer
    RegisterCompareMatchInterrupt(CompareMatchSource1, TimerFrequency_Div1024, 0x80, HeartBeat);
  fc:	23 e5       	ldi	r18, 0x53	; 83
  fe:	30 e0       	ldi	r19, 0x00	; 0
 100:	40 e8       	ldi	r20, 0x80	; 128
 102:	64 e0       	ldi	r22, 0x04	; 4
 104:	80 e0       	ldi	r24, 0x00	; 0
 106:	0e 94 8a 00 	call	0x114	; 0x114 <RegisterCompareMatchInterrupt>

    InitializeStateEventFramework();
 10a:	0e 94 a1 02 	call	0x542	; 0x542 <InitializeStateEventFramework>
    return 0;
 10e:	80 e0       	ldi	r24, 0x00	; 0
 110:	90 e0       	ldi	r25, 0x00	; 0
 112:	08 95       	ret

00000114 <RegisterCompareMatchInterrupt>:
 114:	cf 93       	push	r28
 116:	df 93       	push	r29
 118:	82 30       	cpi	r24, 0x02	; 2
 11a:	48 f4       	brcc	.+18     	; 0x12e <RegisterCompareMatchInterrupt+0x1a>
 11c:	98 2f       	mov	r25, r24
 11e:	93 70       	andi	r25, 0x03	; 3
 120:	cc e3       	ldi	r28, 0x3C	; 60
 122:	d1 e0       	ldi	r29, 0x01	; 1
 124:	ae e6       	ldi	r26, 0x6E	; 110
 126:	b0 e0       	ldi	r27, 0x00	; 0
 128:	e4 e4       	ldi	r30, 0x44	; 68
 12a:	f0 e0       	ldi	r31, 0x00	; 0
 12c:	09 c0       	rjmp	.+18     	; 0x140 <RegisterCompareMatchInterrupt+0x2c>
 12e:	9e ef       	ldi	r25, 0xFE	; 254
 130:	98 0f       	add	r25, r24
 132:	93 70       	andi	r25, 0x03	; 3
 134:	c7 e3       	ldi	r28, 0x37	; 55
 136:	d1 e0       	ldi	r29, 0x01	; 1
 138:	a0 e7       	ldi	r26, 0x70	; 112
 13a:	b0 e0       	ldi	r27, 0x00	; 0
 13c:	e0 eb       	ldi	r30, 0xB0	; 176
 13e:	f0 e0       	ldi	r31, 0x00	; 0
 140:	52 e0       	ldi	r21, 0x02	; 2
 142:	50 83       	st	Z, r21
 144:	c6 0f       	add	r28, r22
 146:	d1 1d       	adc	r29, r1
 148:	58 81       	ld	r21, Y
 14a:	51 83       	std	Z+1, r21	; 0x01
 14c:	33 96       	adiw	r30, 0x03	; 3
 14e:	69 2f       	mov	r22, r25
 150:	70 e0       	ldi	r23, 0x00	; 0
 152:	e6 0f       	add	r30, r22
 154:	f7 1f       	adc	r31, r23
 156:	40 83       	st	Z, r20
 158:	e8 2f       	mov	r30, r24
 15a:	f0 e0       	ldi	r31, 0x00	; 0
 15c:	ee 0f       	add	r30, r30
 15e:	ff 1f       	adc	r31, r31
 160:	e0 53       	subi	r30, 0x30	; 48
 162:	fd 4f       	sbci	r31, 0xFD	; 253
 164:	31 83       	std	Z+1, r19	; 0x01
 166:	20 83       	st	Z, r18
 168:	2c 91       	ld	r18, X
 16a:	6f 5f       	subi	r22, 0xFF	; 255
 16c:	7f 4f       	sbci	r23, 0xFF	; 255
 16e:	81 e0       	ldi	r24, 0x01	; 1
 170:	90 e0       	ldi	r25, 0x00	; 0
 172:	02 c0       	rjmp	.+4      	; 0x178 <RegisterCompareMatchInterrupt+0x64>
 174:	88 0f       	add	r24, r24
 176:	99 1f       	adc	r25, r25
 178:	6a 95       	dec	r22
 17a:	e2 f7       	brpl	.-8      	; 0x174 <RegisterCompareMatchInterrupt+0x60>
 17c:	82 2b       	or	r24, r18
 17e:	8c 93       	st	X, r24
 180:	df 91       	pop	r29
 182:	cf 91       	pop	r28
 184:	08 95       	ret

00000186 <EnterAtomic>:
 186:	f8 94       	cli
 188:	80 91 cf 02 	lds	r24, 0x02CF	; 0x8002cf <_enterAtomicNesting>
 18c:	8f 5f       	subi	r24, 0xFF	; 255
 18e:	80 93 cf 02 	sts	0x02CF, r24	; 0x8002cf <_enterAtomicNesting>
 192:	08 95       	ret

00000194 <LeaveAtomic>:
 194:	80 91 cf 02 	lds	r24, 0x02CF	; 0x8002cf <_enterAtomicNesting>
 198:	88 23       	and	r24, r24
 19a:	31 f0       	breq	.+12     	; 0x1a8 <LeaveAtomic+0x14>
 19c:	81 50       	subi	r24, 0x01	; 1
 19e:	80 93 cf 02 	sts	0x02CF, r24	; 0x8002cf <_enterAtomicNesting>
 1a2:	81 11       	cpse	r24, r1
 1a4:	01 c0       	rjmp	.+2      	; 0x1a8 <LeaveAtomic+0x14>
 1a6:	78 94       	sei
 1a8:	08 95       	ret

000001aa <Usart_Init>:
 1aa:	9b 01       	movw	r18, r22
 1ac:	ac 01       	movw	r20, r24
 1ae:	60 e4       	ldi	r22, 0x40	; 64
 1b0:	72 e4       	ldi	r23, 0x42	; 66
 1b2:	8f e0       	ldi	r24, 0x0F	; 15
 1b4:	90 e0       	ldi	r25, 0x00	; 0
 1b6:	0e 94 a3 04 	call	0x946	; 0x946 <__udivmodsi4>
 1ba:	21 50       	subi	r18, 0x01	; 1
 1bc:	31 09       	sbc	r19, r1
 1be:	e0 ec       	ldi	r30, 0xC0	; 192
 1c0:	f0 e0       	ldi	r31, 0x00	; 0
 1c2:	35 83       	std	Z+5, r19	; 0x05
 1c4:	24 83       	std	Z+4, r18	; 0x04
 1c6:	88 e9       	ldi	r24, 0x98	; 152
 1c8:	81 83       	std	Z+1, r24	; 0x01
 1ca:	8e e0       	ldi	r24, 0x0E	; 14
 1cc:	82 83       	std	Z+2, r24	; 0x02
 1ce:	08 95       	ret

000001d0 <Usart_PutChar>:
 1d0:	cf 93       	push	r28
 1d2:	c8 2f       	mov	r28, r24
 1d4:	0e 94 c3 00 	call	0x186	; 0x186 <EnterAtomic>
 1d8:	80 91 8c 02 	lds	r24, 0x028C	; 0x80028c <USART_txBufferIn>
 1dc:	8f 5f       	subi	r24, 0xFF	; 255
 1de:	8f 71       	andi	r24, 0x1F	; 31
 1e0:	90 91 8b 02 	lds	r25, 0x028B	; 0x80028b <USART_txBufferOut>
 1e4:	89 17       	cp	r24, r25
 1e6:	69 f0       	breq	.+26     	; 0x202 <Usart_PutChar+0x32>
 1e8:	e0 91 8c 02 	lds	r30, 0x028C	; 0x80028c <USART_txBufferIn>
 1ec:	f0 e0       	ldi	r31, 0x00	; 0
 1ee:	e1 57       	subi	r30, 0x71	; 113
 1f0:	fd 4f       	sbci	r31, 0xFD	; 253
 1f2:	c0 83       	st	Z, r28
 1f4:	80 93 8c 02 	sts	0x028C, r24	; 0x80028c <USART_txBufferIn>
 1f8:	e0 ec       	ldi	r30, 0xC0	; 192
 1fa:	f0 e0       	ldi	r31, 0x00	; 0
 1fc:	81 81       	ldd	r24, Z+1	; 0x01
 1fe:	80 62       	ori	r24, 0x20	; 32
 200:	81 83       	std	Z+1, r24	; 0x01
 202:	0e 94 ca 00 	call	0x194	; 0x194 <LeaveAtomic>
 206:	cf 91       	pop	r28
 208:	08 95       	ret

0000020a <SendMessage>:
 20a:	bf 92       	push	r11
 20c:	cf 92       	push	r12
 20e:	df 92       	push	r13
 210:	ef 92       	push	r14
 212:	ff 92       	push	r15
 214:	0f 93       	push	r16
 216:	1f 93       	push	r17
 218:	cf 93       	push	r28
 21a:	df 93       	push	r29
 21c:	b8 2e       	mov	r11, r24
 21e:	d6 2f       	mov	r29, r22
 220:	c4 2e       	mov	r12, r20
 222:	d2 2e       	mov	r13, r18
 224:	c0 91 55 01 	lds	r28, 0x0155	; 0x800155 <_qOut>
 228:	80 91 02 01 	lds	r24, 0x0102	; 0x800102 <_qIn>
 22c:	8c 13       	cpse	r24, r28
 22e:	07 c0       	rjmp	.+14     	; 0x23e <SendMessage+0x34>
 230:	8e ed       	ldi	r24, 0xDE	; 222
 232:	0e 94 e8 00 	call	0x1d0	; 0x1d0 <Usart_PutChar>
 236:	8d ea       	ldi	r24, 0xAD	; 173
 238:	0e 94 e8 00 	call	0x1d0	; 0x1d0 <Usart_PutChar>
 23c:	43 c0       	rjmp	.+134    	; 0x2c4 <SendMessage+0xba>
 23e:	84 ed       	ldi	r24, 0xD4	; 212
 240:	0e 94 e8 00 	call	0x1d0	; 0x1d0 <Usart_PutChar>
 244:	ec 2f       	mov	r30, r28
 246:	f0 e0       	ldi	r31, 0x00	; 0
 248:	ed 5f       	subi	r30, 0xFD	; 253
 24a:	fe 4f       	sbci	r31, 0xFE	; 254
 24c:	e0 80       	ld	r14, Z
 24e:	f1 2c       	mov	r15, r1
 250:	87 01       	movw	r16, r14
 252:	00 0f       	add	r16, r16
 254:	11 1f       	adc	r17, r17
 256:	0e 0d       	add	r16, r14
 258:	1f 1d       	adc	r17, r15
 25a:	00 0f       	add	r16, r16
 25c:	11 1f       	adc	r17, r17
 25e:	0a 5a       	subi	r16, 0xAA	; 170
 260:	1e 4f       	sbci	r17, 0xFE	; 254
 262:	cf 5f       	subi	r28, 0xFF	; 255
 264:	cf 71       	andi	r28, 0x1F	; 31
 266:	c0 93 55 01 	sts	0x0155, r28	; 0x800155 <_qOut>
 26a:	f8 01       	movw	r30, r16
 26c:	b0 82       	st	Z, r11
 26e:	d1 83       	std	Z+1, r29	; 0x01
 270:	c2 82       	std	Z+2, r12	; 0x02
 272:	d3 82       	std	Z+3, r13	; 0x03
 274:	8d 2f       	mov	r24, r29
 276:	80 95       	com	r24
 278:	0e 94 e8 00 	call	0x1d0	; 0x1d0 <Usart_PutChar>
 27c:	f8 01       	movw	r30, r16
 27e:	20 81       	ld	r18, Z
 280:	c3 e2       	ldi	r28, 0x23	; 35
 282:	d1 e0       	ldi	r29, 0x01	; 1
 284:	fe 01       	movw	r30, r28
 286:	02 c0       	rjmp	.+4      	; 0x28c <SendMessage+0x82>
 288:	ef 01       	movw	r28, r30
 28a:	fc 01       	movw	r30, r24
 28c:	80 81       	ld	r24, Z
 28e:	82 17       	cp	r24, r18
 290:	30 f0       	brcs	.+12     	; 0x29e <SendMessage+0x94>
 292:	84 81       	ldd	r24, Z+4	; 0x04
 294:	95 81       	ldd	r25, Z+5	; 0x05
 296:	31 e0       	ldi	r19, 0x01	; 1
 298:	83 32       	cpi	r24, 0x23	; 35
 29a:	93 07       	cpc	r25, r19
 29c:	a9 f7       	brne	.-22     	; 0x288 <SendMessage+0x7e>
 29e:	0e 94 c3 00 	call	0x186	; 0x186 <EnterAtomic>
 2a2:	8c 81       	ldd	r24, Y+4	; 0x04
 2a4:	9d 81       	ldd	r25, Y+5	; 0x05
 2a6:	f7 01       	movw	r30, r14
 2a8:	ee 0f       	add	r30, r30
 2aa:	ff 1f       	adc	r31, r31
 2ac:	ee 0d       	add	r30, r14
 2ae:	ff 1d       	adc	r31, r15
 2b0:	ee 0f       	add	r30, r30
 2b2:	ff 1f       	adc	r31, r31
 2b4:	ea 5a       	subi	r30, 0xAA	; 170
 2b6:	fe 4f       	sbci	r31, 0xFE	; 254
 2b8:	95 83       	std	Z+5, r25	; 0x05
 2ba:	84 83       	std	Z+4, r24	; 0x04
 2bc:	1d 83       	std	Y+5, r17	; 0x05
 2be:	0c 83       	std	Y+4, r16	; 0x04
 2c0:	0e 94 ca 00 	call	0x194	; 0x194 <LeaveAtomic>
 2c4:	df 91       	pop	r29
 2c6:	cf 91       	pop	r28
 2c8:	1f 91       	pop	r17
 2ca:	0f 91       	pop	r16
 2cc:	ff 90       	pop	r15
 2ce:	ef 90       	pop	r14
 2d0:	df 90       	pop	r13
 2d2:	cf 90       	pop	r12
 2d4:	bf 90       	pop	r11
 2d6:	08 95       	ret

000002d8 <ProcessMessage>:
 2d8:	ff 92       	push	r15
 2da:	0f 93       	push	r16
 2dc:	1f 93       	push	r17
 2de:	cf 93       	push	r28
 2e0:	df 93       	push	r29
 2e2:	c8 2f       	mov	r28, r24
 2e4:	8b 01       	movw	r16, r22
 2e6:	d4 2f       	mov	r29, r20
 2e8:	81 ed       	ldi	r24, 0xD1	; 209
 2ea:	0e 94 e8 00 	call	0x1d0	; 0x1d0 <Usart_PutChar>
 2ee:	80 91 1a 02 	lds	r24, 0x021A	; 0x80021a <_avrPoolOut>
 2f2:	90 91 2e 01 	lds	r25, 0x012E	; 0x80012e <_avrPoolIn>
 2f6:	89 17       	cp	r24, r25
 2f8:	99 f1       	breq	.+102    	; 0x360 <ProcessMessage+0x88>
 2fa:	e8 2f       	mov	r30, r24
 2fc:	f0 e0       	ldi	r31, 0x00	; 0
 2fe:	e1 5d       	subi	r30, 0xD1	; 209
 300:	fe 4f       	sbci	r31, 0xFE	; 254
 302:	f0 80       	ld	r15, Z
 304:	8f 5f       	subi	r24, 0xFF	; 255
 306:	87 70       	andi	r24, 0x07	; 7
 308:	80 93 1a 02 	sts	0x021A, r24	; 0x80021a <_avrPoolOut>
 30c:	85 ed       	ldi	r24, 0xD5	; 213
 30e:	0e 94 e8 00 	call	0x1d0	; 0x1d0 <Usart_PutChar>
 312:	8f 2d       	mov	r24, r15
 314:	0e 94 e8 00 	call	0x1d0	; 0x1d0 <Usart_PutChar>
 318:	8c 2f       	mov	r24, r28
 31a:	80 95       	com	r24
 31c:	0e 94 e8 00 	call	0x1d0	; 0x1d0 <Usart_PutChar>
 320:	2f 2d       	mov	r18, r15
 322:	30 e0       	ldi	r19, 0x00	; 0
 324:	22 0f       	add	r18, r18
 326:	33 1f       	adc	r19, r19
 328:	c9 01       	movw	r24, r18
 32a:	88 0f       	add	r24, r24
 32c:	99 1f       	adc	r25, r25
 32e:	88 0f       	add	r24, r24
 330:	99 1f       	adc	r25, r25
 332:	88 0f       	add	r24, r24
 334:	99 1f       	adc	r25, r25
 336:	82 1b       	sub	r24, r18
 338:	93 0b       	sbc	r25, r19
 33a:	fc 01       	movw	r30, r24
 33c:	e5 5e       	subi	r30, 0xE5	; 229
 33e:	fd 4f       	sbci	r31, 0xFD	; 253
 340:	c0 83       	st	Z, r28
 342:	d1 83       	std	Z+1, r29	; 0x01
 344:	4d 2f       	mov	r20, r29
 346:	50 e0       	ldi	r21, 0x00	; 0
 348:	b8 01       	movw	r22, r16
 34a:	83 5e       	subi	r24, 0xE3	; 227
 34c:	9d 4f       	sbci	r25, 0xFD	; 253
 34e:	0e 94 c5 04 	call	0x98a	; 0x98a <memcpy>
 352:	6c 2f       	mov	r22, r28
 354:	60 68       	ori	r22, 0x80	; 128
 356:	20 e0       	ldi	r18, 0x00	; 0
 358:	4f 2d       	mov	r20, r15
 35a:	80 e0       	ldi	r24, 0x00	; 0
 35c:	0e 94 05 01 	call	0x20a	; 0x20a <SendMessage>
 360:	df 91       	pop	r29
 362:	cf 91       	pop	r28
 364:	1f 91       	pop	r17
 366:	0f 91       	pop	r16
 368:	ff 90       	pop	r15
 36a:	08 95       	ret

0000036c <HandleMessage>:
 36c:	90 91 54 01 	lds	r25, 0x0154	; 0x800154 <msgType.2106>
 370:	91 11       	cpse	r25, r1
 372:	05 c0       	rjmp	.+10     	; 0x37e <HandleMessage+0x12>
 374:	80 93 54 01 	sts	0x0154, r24	; 0x800154 <msgType.2106>
 378:	10 92 53 01 	sts	0x0153, r1	; 0x800153 <msgLen.2107>
 37c:	08 95       	ret
 37e:	40 91 53 01 	lds	r20, 0x0153	; 0x800153 <msgLen.2107>
 382:	41 11       	cpse	r20, r1
 384:	06 c0       	rjmp	.+12     	; 0x392 <HandleMessage+0x26>
 386:	82 50       	subi	r24, 0x02	; 2
 388:	80 93 53 01 	sts	0x0153, r24	; 0x800153 <msgLen.2107>
 38c:	10 92 52 01 	sts	0x0152, r1	; 0x800152 <bufferIndex.2105>
 390:	08 95       	ret
 392:	e0 91 52 01 	lds	r30, 0x0152	; 0x800152 <bufferIndex.2105>
 396:	e4 17       	cp	r30, r20
 398:	98 f4       	brcc	.+38     	; 0x3c0 <HandleMessage+0x54>
 39a:	21 e0       	ldi	r18, 0x01	; 1
 39c:	2e 0f       	add	r18, r30
 39e:	20 93 52 01 	sts	0x0152, r18	; 0x800152 <bufferIndex.2105>
 3a2:	f0 e0       	ldi	r31, 0x00	; 0
 3a4:	ec 5b       	subi	r30, 0xBC	; 188
 3a6:	fe 4f       	sbci	r31, 0xFE	; 254
 3a8:	80 83       	st	Z, r24
 3aa:	42 13       	cpse	r20, r18
 3ac:	09 c0       	rjmp	.+18     	; 0x3c0 <HandleMessage+0x54>
 3ae:	64 e4       	ldi	r22, 0x44	; 68
 3b0:	71 e0       	ldi	r23, 0x01	; 1
 3b2:	89 2f       	mov	r24, r25
 3b4:	0e 94 6c 01 	call	0x2d8	; 0x2d8 <ProcessMessage>
 3b8:	10 92 54 01 	sts	0x0154, r1	; 0x800154 <msgType.2106>
 3bc:	10 92 52 01 	sts	0x0152, r1	; 0x800152 <bufferIndex.2105>
 3c0:	08 95       	ret

000003c2 <GetMessage>:
 3c2:	cf 93       	push	r28
 3c4:	df 93       	push	r29
 3c6:	c0 91 27 01 	lds	r28, 0x0127	; 0x800127 <_root+0x4>
 3ca:	d0 91 28 01 	lds	r29, 0x0128	; 0x800128 <_root+0x5>
 3ce:	21 e0       	ldi	r18, 0x01	; 1
 3d0:	c3 32       	cpi	r28, 0x23	; 35
 3d2:	d2 07       	cpc	r29, r18
 3d4:	b9 f1       	breq	.+110    	; 0x444 <__LOCK_REGION_LENGTH__+0x44>
 3d6:	26 e0       	ldi	r18, 0x06	; 6
 3d8:	fe 01       	movw	r30, r28
 3da:	dc 01       	movw	r26, r24
 3dc:	01 90       	ld	r0, Z+
 3de:	0d 92       	st	X+, r0
 3e0:	2a 95       	dec	r18
 3e2:	e1 f7       	brne	.-8      	; 0x3dc <GetMessage+0x1a>
 3e4:	fc 01       	movw	r30, r24
 3e6:	15 82       	std	Z+5, r1	; 0x05
 3e8:	14 82       	std	Z+4, r1	; 0x04
 3ea:	0e 94 c3 00 	call	0x186	; 0x186 <EnterAtomic>
 3ee:	80 91 02 01 	lds	r24, 0x0102	; 0x800102 <_qIn>
 3f2:	e8 2f       	mov	r30, r24
 3f4:	f0 e0       	ldi	r31, 0x00	; 0
 3f6:	ed 5f       	subi	r30, 0xFD	; 253
 3f8:	fe 4f       	sbci	r31, 0xFE	; 254
 3fa:	9e 01       	movw	r18, r28
 3fc:	26 55       	subi	r18, 0x56	; 86
 3fe:	31 40       	sbci	r19, 0x01	; 1
 400:	35 95       	asr	r19
 402:	27 95       	ror	r18
 404:	6b ea       	ldi	r22, 0xAB	; 171
 406:	7a ea       	ldi	r23, 0xAA	; 170
 408:	26 9f       	mul	r18, r22
 40a:	a0 01       	movw	r20, r0
 40c:	27 9f       	mul	r18, r23
 40e:	50 0d       	add	r21, r0
 410:	36 9f       	mul	r19, r22
 412:	50 0d       	add	r21, r0
 414:	11 24       	eor	r1, r1
 416:	40 83       	st	Z, r20
 418:	2c 81       	ldd	r18, Y+4	; 0x04
 41a:	3d 81       	ldd	r19, Y+5	; 0x05
 41c:	30 93 28 01 	sts	0x0128, r19	; 0x800128 <_root+0x5>
 420:	20 93 27 01 	sts	0x0127, r18	; 0x800127 <_root+0x4>
 424:	96 e0       	ldi	r25, 0x06	; 6
 426:	fe 01       	movw	r30, r28
 428:	11 92       	st	Z+, r1
 42a:	9a 95       	dec	r25
 42c:	e9 f7       	brne	.-6      	; 0x428 <__LOCK_REGION_LENGTH__+0x28>
 42e:	8f 5f       	subi	r24, 0xFF	; 255
 430:	8f 71       	andi	r24, 0x1F	; 31
 432:	80 93 02 01 	sts	0x0102, r24	; 0x800102 <_qIn>
 436:	0e 94 ca 00 	call	0x194	; 0x194 <LeaveAtomic>
 43a:	83 ed       	ldi	r24, 0xD3	; 211
 43c:	0e 94 e8 00 	call	0x1d0	; 0x1d0 <Usart_PutChar>
 440:	81 e0       	ldi	r24, 0x01	; 1
 442:	01 c0       	rjmp	.+2      	; 0x446 <__LOCK_REGION_LENGTH__+0x46>
 444:	80 e0       	ldi	r24, 0x00	; 0
 446:	df 91       	pop	r29
 448:	cf 91       	pop	r28
 44a:	08 95       	ret

0000044c <DispatchEvent>:
 44c:	ff 92       	push	r15
 44e:	0f 93       	push	r16
 450:	1f 93       	push	r17
 452:	cf 93       	push	r28
 454:	df 93       	push	r29
 456:	00 d0       	rcall	.+0      	; 0x458 <DispatchEvent+0xc>
 458:	00 d0       	rcall	.+0      	; 0x45a <DispatchEvent+0xe>
 45a:	00 d0       	rcall	.+0      	; 0x45c <DispatchEvent+0x10>
 45c:	cd b7       	in	r28, 0x3d	; 61
 45e:	de b7       	in	r29, 0x3e	; 62
 460:	ce 01       	movw	r24, r28
 462:	01 96       	adiw	r24, 0x01	; 1
 464:	26 e0       	ldi	r18, 0x06	; 6
 466:	dc 01       	movw	r26, r24
 468:	1d 92       	st	X+, r1
 46a:	2a 95       	dec	r18
 46c:	e9 f7       	brne	.-6      	; 0x468 <DispatchEvent+0x1c>
 46e:	0e 94 e1 01 	call	0x3c2	; 0x3c2 <GetMessage>
 472:	88 23       	and	r24, r24
 474:	09 f4       	brne	.+2      	; 0x478 <DispatchEvent+0x2c>
 476:	59 c0       	rjmp	.+178    	; 0x52a <DispatchEvent+0xde>
 478:	82 ed       	ldi	r24, 0xD2	; 210
 47a:	0e 94 e8 00 	call	0x1d0	; 0x1d0 <Usart_PutChar>
 47e:	8a 81       	ldd	r24, Y+2	; 0x02
 480:	88 23       	and	r24, r24
 482:	5c f5       	brge	.+86     	; 0x4da <DispatchEvent+0x8e>
 484:	fb 80       	ldd	r15, Y+3	; 0x03
 486:	8f 2d       	mov	r24, r15
 488:	0e 94 e8 00 	call	0x1d0	; 0x1d0 <Usart_PutChar>
 48c:	8f 2d       	mov	r24, r15
 48e:	90 e0       	ldi	r25, 0x00	; 0
 490:	88 0f       	add	r24, r24
 492:	99 1f       	adc	r25, r25
 494:	8c 01       	movw	r16, r24
 496:	00 0f       	add	r16, r16
 498:	11 1f       	adc	r17, r17
 49a:	00 0f       	add	r16, r16
 49c:	11 1f       	adc	r17, r17
 49e:	00 0f       	add	r16, r16
 4a0:	11 1f       	adc	r17, r17
 4a2:	08 1b       	sub	r16, r24
 4a4:	19 0b       	sbc	r17, r25
 4a6:	05 5e       	subi	r16, 0xE5	; 229
 4a8:	1d 4f       	sbci	r17, 0xFD	; 253
 4aa:	f8 01       	movw	r30, r16
 4ac:	80 81       	ld	r24, Z
 4ae:	80 95       	com	r24
 4b0:	0e 94 e8 00 	call	0x1d0	; 0x1d0 <Usart_PutChar>
 4b4:	e0 91 00 01 	lds	r30, 0x0100	; 0x800100 <__data_start>
 4b8:	f0 91 01 01 	lds	r31, 0x0101	; 0x800101 <__data_start+0x1>
 4bc:	c8 01       	movw	r24, r16
 4be:	09 95       	icall
 4c0:	80 91 2e 01 	lds	r24, 0x012E	; 0x80012e <_avrPoolIn>
 4c4:	e8 2f       	mov	r30, r24
 4c6:	f0 e0       	ldi	r31, 0x00	; 0
 4c8:	e1 5d       	subi	r30, 0xD1	; 209
 4ca:	fe 4f       	sbci	r31, 0xFE	; 254
 4cc:	f0 82       	st	Z, r15
 4ce:	8f 5f       	subi	r24, 0xFF	; 255
 4d0:	87 70       	andi	r24, 0x07	; 7
 4d2:	80 93 2e 01 	sts	0x012E, r24	; 0x80012e <_avrPoolIn>
 4d6:	81 e0       	ldi	r24, 0x01	; 1
 4d8:	28 c0       	rjmp	.+80     	; 0x52a <DispatchEvent+0xde>
 4da:	00 91 29 01 	lds	r16, 0x0129	; 0x800129 <_anchor>
 4de:	10 91 2a 01 	lds	r17, 0x012A	; 0x80012a <_anchor+0x1>
 4e2:	81 e0       	ldi	r24, 0x01	; 1
 4e4:	90 e0       	ldi	r25, 0x00	; 0
 4e6:	09 80       	ldd	r0, Y+1	; 0x01
 4e8:	02 c0       	rjmp	.+4      	; 0x4ee <DispatchEvent+0xa2>
 4ea:	88 0f       	add	r24, r24
 4ec:	99 1f       	adc	r25, r25
 4ee:	0a 94       	dec	r0
 4f0:	e2 f7       	brpl	.-8      	; 0x4ea <DispatchEvent+0x9e>
 4f2:	f8 2e       	mov	r15, r24
 4f4:	f1 e0       	ldi	r31, 0x01	; 1
 4f6:	09 32       	cpi	r16, 0x29	; 41
 4f8:	1f 07       	cpc	r17, r31
 4fa:	b1 f0       	breq	.+44     	; 0x528 <DispatchEvent+0xdc>
 4fc:	d8 01       	movw	r26, r16
 4fe:	12 96       	adiw	r26, 0x02	; 2
 500:	8c 91       	ld	r24, X
 502:	12 97       	sbiw	r26, 0x02	; 2
 504:	8f 21       	and	r24, r15
 506:	39 f0       	breq	.+14     	; 0x516 <DispatchEvent+0xca>
 508:	13 96       	adiw	r26, 0x03	; 3
 50a:	ed 91       	ld	r30, X+
 50c:	fc 91       	ld	r31, X
 50e:	14 97       	sbiw	r26, 0x04	; 4
 510:	ce 01       	movw	r24, r28
 512:	01 96       	adiw	r24, 0x01	; 1
 514:	09 95       	icall
 516:	f8 01       	movw	r30, r16
 518:	00 81       	ld	r16, Z
 51a:	11 81       	ldd	r17, Z+1	; 0x01
 51c:	f1 e0       	ldi	r31, 0x01	; 1
 51e:	09 32       	cpi	r16, 0x29	; 41
 520:	1f 07       	cpc	r17, r31
 522:	61 f7       	brne	.-40     	; 0x4fc <DispatchEvent+0xb0>
 524:	81 e0       	ldi	r24, 0x01	; 1
 526:	01 c0       	rjmp	.+2      	; 0x52a <DispatchEvent+0xde>
 528:	81 e0       	ldi	r24, 0x01	; 1
 52a:	26 96       	adiw	r28, 0x06	; 6
 52c:	0f b6       	in	r0, 0x3f	; 63
 52e:	f8 94       	cli
 530:	de bf       	out	0x3e, r29	; 62
 532:	0f be       	out	0x3f, r0	; 63
 534:	cd bf       	out	0x3d, r28	; 61
 536:	df 91       	pop	r29
 538:	cf 91       	pop	r28
 53a:	1f 91       	pop	r17
 53c:	0f 91       	pop	r16
 53e:	ff 90       	pop	r15
 540:	08 95       	ret

00000542 <InitializeStateEventFramework>:
 542:	8a ec       	ldi	r24, 0xCA	; 202
 544:	0e 94 e8 00 	call	0x1d0	; 0x1d0 <Usart_PutChar>
 548:	8e ef       	ldi	r24, 0xFE	; 254
 54a:	0e 94 e8 00 	call	0x1d0	; 0x1d0 <Usart_PutChar>
 54e:	0e 94 26 02 	call	0x44c	; 0x44c <DispatchEvent>
 552:	90 91 8d 02 	lds	r25, 0x028D	; 0x80028d <USART_rxBufferOut>
 556:	80 91 8e 02 	lds	r24, 0x028E	; 0x80028e <USART_rxBufferIn>
 55a:	98 17       	cp	r25, r24
 55c:	c1 f3       	breq	.-16     	; 0x54e <InitializeStateEventFramework+0xc>
 55e:	0e 94 c3 00 	call	0x186	; 0x186 <EnterAtomic>
 562:	e0 91 8d 02 	lds	r30, 0x028D	; 0x80028d <USART_rxBufferOut>
 566:	81 e0       	ldi	r24, 0x01	; 1
 568:	8e 0f       	add	r24, r30
 56a:	80 93 8d 02 	sts	0x028D, r24	; 0x80028d <USART_rxBufferOut>
 56e:	f0 e0       	ldi	r31, 0x00	; 0
 570:	e1 55       	subi	r30, 0x51	; 81
 572:	fd 4f       	sbci	r31, 0xFD	; 253
 574:	c0 81       	ld	r28, Z
 576:	80 91 8d 02 	lds	r24, 0x028D	; 0x80028d <USART_rxBufferOut>
 57a:	8f 71       	andi	r24, 0x1F	; 31
 57c:	80 93 8d 02 	sts	0x028D, r24	; 0x80028d <USART_rxBufferOut>
 580:	0e 94 ca 00 	call	0x194	; 0x194 <LeaveAtomic>
 584:	8c 2f       	mov	r24, r28
 586:	0e 94 b6 01 	call	0x36c	; 0x36c <HandleMessage>
 58a:	90 91 8d 02 	lds	r25, 0x028D	; 0x80028d <USART_rxBufferOut>
 58e:	80 91 8e 02 	lds	r24, 0x028E	; 0x80028e <USART_rxBufferIn>
 592:	98 13       	cpse	r25, r24
 594:	e4 cf       	rjmp	.-56     	; 0x55e <InitializeStateEventFramework+0x1c>
 596:	db cf       	rjmp	.-74     	; 0x54e <InitializeStateEventFramework+0xc>

00000598 <__vector_19>:
 598:	1f 92       	push	r1
 59a:	0f 92       	push	r0
 59c:	0f b6       	in	r0, 0x3f	; 63
 59e:	0f 92       	push	r0
 5a0:	11 24       	eor	r1, r1
 5a2:	8f 93       	push	r24
 5a4:	9f 93       	push	r25
 5a6:	ef 93       	push	r30
 5a8:	ff 93       	push	r31
 5aa:	90 91 8b 02 	lds	r25, 0x028B	; 0x80028b <USART_txBufferOut>
 5ae:	80 91 8c 02 	lds	r24, 0x028C	; 0x80028c <USART_txBufferIn>
 5b2:	98 17       	cp	r25, r24
 5b4:	91 f0       	breq	.+36     	; 0x5da <__vector_19+0x42>
 5b6:	e0 91 8b 02 	lds	r30, 0x028B	; 0x80028b <USART_txBufferOut>
 5ba:	81 e0       	ldi	r24, 0x01	; 1
 5bc:	8e 0f       	add	r24, r30
 5be:	80 93 8b 02 	sts	0x028B, r24	; 0x80028b <USART_txBufferOut>
 5c2:	f0 e0       	ldi	r31, 0x00	; 0
 5c4:	e1 57       	subi	r30, 0x71	; 113
 5c6:	fd 4f       	sbci	r31, 0xFD	; 253
 5c8:	80 81       	ld	r24, Z
 5ca:	80 93 c6 00 	sts	0x00C6, r24	; 0x8000c6 <__TEXT_REGION_LENGTH__+0x7e00c6>
 5ce:	80 91 8b 02 	lds	r24, 0x028B	; 0x80028b <USART_txBufferOut>
 5d2:	8f 71       	andi	r24, 0x1F	; 31
 5d4:	80 93 8b 02 	sts	0x028B, r24	; 0x80028b <USART_txBufferOut>
 5d8:	05 c0       	rjmp	.+10     	; 0x5e4 <__vector_19+0x4c>
 5da:	e0 ec       	ldi	r30, 0xC0	; 192
 5dc:	f0 e0       	ldi	r31, 0x00	; 0
 5de:	81 81       	ldd	r24, Z+1	; 0x01
 5e0:	8f 7d       	andi	r24, 0xDF	; 223
 5e2:	81 83       	std	Z+1, r24	; 0x01
 5e4:	ff 91       	pop	r31
 5e6:	ef 91       	pop	r30
 5e8:	9f 91       	pop	r25
 5ea:	8f 91       	pop	r24
 5ec:	0f 90       	pop	r0
 5ee:	0f be       	out	0x3f, r0	; 63
 5f0:	0f 90       	pop	r0
 5f2:	1f 90       	pop	r1
 5f4:	18 95       	reti

000005f6 <__vector_18>:
 5f6:	1f 92       	push	r1
 5f8:	0f 92       	push	r0
 5fa:	0f b6       	in	r0, 0x3f	; 63
 5fc:	0f 92       	push	r0
 5fe:	11 24       	eor	r1, r1
 600:	2f 93       	push	r18
 602:	8f 93       	push	r24
 604:	9f 93       	push	r25
 606:	af 93       	push	r26
 608:	bf 93       	push	r27
 60a:	ef 93       	push	r30
 60c:	ff 93       	push	r31
 60e:	e0 ec       	ldi	r30, 0xC0	; 192
 610:	f0 e0       	ldi	r31, 0x00	; 0
 612:	11 c0       	rjmp	.+34     	; 0x636 <__vector_18+0x40>
 614:	26 81       	ldd	r18, Z+6	; 0x06
 616:	80 91 8e 02 	lds	r24, 0x028E	; 0x80028e <USART_rxBufferIn>
 61a:	8f 5f       	subi	r24, 0xFF	; 255
 61c:	8f 71       	andi	r24, 0x1F	; 31
 61e:	90 91 8d 02 	lds	r25, 0x028D	; 0x80028d <USART_rxBufferOut>
 622:	89 17       	cp	r24, r25
 624:	41 f0       	breq	.+16     	; 0x636 <__vector_18+0x40>
 626:	a0 91 8e 02 	lds	r26, 0x028E	; 0x80028e <USART_rxBufferIn>
 62a:	b0 e0       	ldi	r27, 0x00	; 0
 62c:	a1 55       	subi	r26, 0x51	; 81
 62e:	bd 4f       	sbci	r27, 0xFD	; 253
 630:	2c 93       	st	X, r18
 632:	80 93 8e 02 	sts	0x028E, r24	; 0x80028e <USART_rxBufferIn>
 636:	80 81       	ld	r24, Z
 638:	88 23       	and	r24, r24
 63a:	64 f3       	brlt	.-40     	; 0x614 <__vector_18+0x1e>
 63c:	ff 91       	pop	r31
 63e:	ef 91       	pop	r30
 640:	bf 91       	pop	r27
 642:	af 91       	pop	r26
 644:	9f 91       	pop	r25
 646:	8f 91       	pop	r24
 648:	2f 91       	pop	r18
 64a:	0f 90       	pop	r0
 64c:	0f be       	out	0x3f, r0	; 63
 64e:	0f 90       	pop	r0
 650:	1f 90       	pop	r1
 652:	18 95       	reti

00000654 <__vector_1>:
 654:	1f 92       	push	r1
 656:	0f 92       	push	r0
 658:	0f b6       	in	r0, 0x3f	; 63
 65a:	0f 92       	push	r0
 65c:	11 24       	eor	r1, r1
 65e:	2f 93       	push	r18
 660:	3f 93       	push	r19
 662:	4f 93       	push	r20
 664:	5f 93       	push	r21
 666:	6f 93       	push	r22
 668:	7f 93       	push	r23
 66a:	8f 93       	push	r24
 66c:	9f 93       	push	r25
 66e:	af 93       	push	r26
 670:	bf 93       	push	r27
 672:	ef 93       	push	r30
 674:	ff 93       	push	r31
 676:	e0 91 d8 02 	lds	r30, 0x02D8	; 0x8002d8 <_extIntHandler>
 67a:	f0 91 d9 02 	lds	r31, 0x02D9	; 0x8002d9 <_extIntHandler+0x1>
 67e:	30 97       	sbiw	r30, 0x00	; 0
 680:	09 f0       	breq	.+2      	; 0x684 <__vector_1+0x30>
 682:	09 95       	icall
 684:	ff 91       	pop	r31
 686:	ef 91       	pop	r30
 688:	bf 91       	pop	r27
 68a:	af 91       	pop	r26
 68c:	9f 91       	pop	r25
 68e:	8f 91       	pop	r24
 690:	7f 91       	pop	r23
 692:	6f 91       	pop	r22
 694:	5f 91       	pop	r21
 696:	4f 91       	pop	r20
 698:	3f 91       	pop	r19
 69a:	2f 91       	pop	r18
 69c:	0f 90       	pop	r0
 69e:	0f be       	out	0x3f, r0	; 63
 6a0:	0f 90       	pop	r0
 6a2:	1f 90       	pop	r1
 6a4:	18 95       	reti

000006a6 <__vector_2>:
 6a6:	1f 92       	push	r1
 6a8:	0f 92       	push	r0
 6aa:	0f b6       	in	r0, 0x3f	; 63
 6ac:	0f 92       	push	r0
 6ae:	11 24       	eor	r1, r1
 6b0:	2f 93       	push	r18
 6b2:	3f 93       	push	r19
 6b4:	4f 93       	push	r20
 6b6:	5f 93       	push	r21
 6b8:	6f 93       	push	r22
 6ba:	7f 93       	push	r23
 6bc:	8f 93       	push	r24
 6be:	9f 93       	push	r25
 6c0:	af 93       	push	r26
 6c2:	bf 93       	push	r27
 6c4:	ef 93       	push	r30
 6c6:	ff 93       	push	r31
 6c8:	e0 91 da 02 	lds	r30, 0x02DA	; 0x8002da <_extIntHandler+0x2>
 6cc:	f0 91 db 02 	lds	r31, 0x02DB	; 0x8002db <_extIntHandler+0x3>
 6d0:	30 97       	sbiw	r30, 0x00	; 0
 6d2:	09 f0       	breq	.+2      	; 0x6d6 <__vector_2+0x30>
 6d4:	09 95       	icall
 6d6:	ff 91       	pop	r31
 6d8:	ef 91       	pop	r30
 6da:	bf 91       	pop	r27
 6dc:	af 91       	pop	r26
 6de:	9f 91       	pop	r25
 6e0:	8f 91       	pop	r24
 6e2:	7f 91       	pop	r23
 6e4:	6f 91       	pop	r22
 6e6:	5f 91       	pop	r21
 6e8:	4f 91       	pop	r20
 6ea:	3f 91       	pop	r19
 6ec:	2f 91       	pop	r18
 6ee:	0f 90       	pop	r0
 6f0:	0f be       	out	0x3f, r0	; 63
 6f2:	0f 90       	pop	r0
 6f4:	1f 90       	pop	r1
 6f6:	18 95       	reti

000006f8 <__vector_14>:
 6f8:	1f 92       	push	r1
 6fa:	0f 92       	push	r0
 6fc:	0f b6       	in	r0, 0x3f	; 63
 6fe:	0f 92       	push	r0
 700:	11 24       	eor	r1, r1
 702:	2f 93       	push	r18
 704:	3f 93       	push	r19
 706:	4f 93       	push	r20
 708:	5f 93       	push	r21
 70a:	6f 93       	push	r22
 70c:	7f 93       	push	r23
 70e:	8f 93       	push	r24
 710:	9f 93       	push	r25
 712:	af 93       	push	r26
 714:	bf 93       	push	r27
 716:	ef 93       	push	r30
 718:	ff 93       	push	r31
 71a:	e0 91 d0 02 	lds	r30, 0x02D0	; 0x8002d0 <_compareMatchHandler>
 71e:	f0 91 d1 02 	lds	r31, 0x02D1	; 0x8002d1 <_compareMatchHandler+0x1>
 722:	30 97       	sbiw	r30, 0x00	; 0
 724:	09 f0       	breq	.+2      	; 0x728 <__vector_14+0x30>
 726:	09 95       	icall
 728:	ff 91       	pop	r31
 72a:	ef 91       	pop	r30
 72c:	bf 91       	pop	r27
 72e:	af 91       	pop	r26
 730:	9f 91       	pop	r25
 732:	8f 91       	pop	r24
 734:	7f 91       	pop	r23
 736:	6f 91       	pop	r22
 738:	5f 91       	pop	r21
 73a:	4f 91       	pop	r20
 73c:	3f 91       	pop	r19
 73e:	2f 91       	pop	r18
 740:	0f 90       	pop	r0
 742:	0f be       	out	0x3f, r0	; 63
 744:	0f 90       	pop	r0
 746:	1f 90       	pop	r1
 748:	18 95       	reti

0000074a <__vector_15>:
 74a:	1f 92       	push	r1
 74c:	0f 92       	push	r0
 74e:	0f b6       	in	r0, 0x3f	; 63
 750:	0f 92       	push	r0
 752:	11 24       	eor	r1, r1
 754:	2f 93       	push	r18
 756:	3f 93       	push	r19
 758:	4f 93       	push	r20
 75a:	5f 93       	push	r21
 75c:	6f 93       	push	r22
 75e:	7f 93       	push	r23
 760:	8f 93       	push	r24
 762:	9f 93       	push	r25
 764:	af 93       	push	r26
 766:	bf 93       	push	r27
 768:	ef 93       	push	r30
 76a:	ff 93       	push	r31
 76c:	e0 91 d2 02 	lds	r30, 0x02D2	; 0x8002d2 <_compareMatchHandler+0x2>
 770:	f0 91 d3 02 	lds	r31, 0x02D3	; 0x8002d3 <_compareMatchHandler+0x3>
 774:	30 97       	sbiw	r30, 0x00	; 0
 776:	09 f0       	breq	.+2      	; 0x77a <__vector_15+0x30>
 778:	09 95       	icall
 77a:	ff 91       	pop	r31
 77c:	ef 91       	pop	r30
 77e:	bf 91       	pop	r27
 780:	af 91       	pop	r26
 782:	9f 91       	pop	r25
 784:	8f 91       	pop	r24
 786:	7f 91       	pop	r23
 788:	6f 91       	pop	r22
 78a:	5f 91       	pop	r21
 78c:	4f 91       	pop	r20
 78e:	3f 91       	pop	r19
 790:	2f 91       	pop	r18
 792:	0f 90       	pop	r0
 794:	0f be       	out	0x3f, r0	; 63
 796:	0f 90       	pop	r0
 798:	1f 90       	pop	r1
 79a:	18 95       	reti

0000079c <__vector_7>:
 79c:	1f 92       	push	r1
 79e:	0f 92       	push	r0
 7a0:	0f b6       	in	r0, 0x3f	; 63
 7a2:	0f 92       	push	r0
 7a4:	11 24       	eor	r1, r1
 7a6:	2f 93       	push	r18
 7a8:	3f 93       	push	r19
 7aa:	4f 93       	push	r20
 7ac:	5f 93       	push	r21
 7ae:	6f 93       	push	r22
 7b0:	7f 93       	push	r23
 7b2:	8f 93       	push	r24
 7b4:	9f 93       	push	r25
 7b6:	af 93       	push	r26
 7b8:	bf 93       	push	r27
 7ba:	ef 93       	push	r30
 7bc:	ff 93       	push	r31
 7be:	e0 91 d4 02 	lds	r30, 0x02D4	; 0x8002d4 <_compareMatchHandler+0x4>
 7c2:	f0 91 d5 02 	lds	r31, 0x02D5	; 0x8002d5 <_compareMatchHandler+0x5>
 7c6:	30 97       	sbiw	r30, 0x00	; 0
 7c8:	09 f0       	breq	.+2      	; 0x7cc <__vector_7+0x30>
 7ca:	09 95       	icall
 7cc:	ff 91       	pop	r31
 7ce:	ef 91       	pop	r30
 7d0:	bf 91       	pop	r27
 7d2:	af 91       	pop	r26
 7d4:	9f 91       	pop	r25
 7d6:	8f 91       	pop	r24
 7d8:	7f 91       	pop	r23
 7da:	6f 91       	pop	r22
 7dc:	5f 91       	pop	r21
 7de:	4f 91       	pop	r20
 7e0:	3f 91       	pop	r19
 7e2:	2f 91       	pop	r18
 7e4:	0f 90       	pop	r0
 7e6:	0f be       	out	0x3f, r0	; 63
 7e8:	0f 90       	pop	r0
 7ea:	1f 90       	pop	r1
 7ec:	18 95       	reti

000007ee <__vector_8>:
 7ee:	1f 92       	push	r1
 7f0:	0f 92       	push	r0
 7f2:	0f b6       	in	r0, 0x3f	; 63
 7f4:	0f 92       	push	r0
 7f6:	11 24       	eor	r1, r1
 7f8:	2f 93       	push	r18
 7fa:	3f 93       	push	r19
 7fc:	4f 93       	push	r20
 7fe:	5f 93       	push	r21
 800:	6f 93       	push	r22
 802:	7f 93       	push	r23
 804:	8f 93       	push	r24
 806:	9f 93       	push	r25
 808:	af 93       	push	r26
 80a:	bf 93       	push	r27
 80c:	ef 93       	push	r30
 80e:	ff 93       	push	r31
 810:	e0 91 d6 02 	lds	r30, 0x02D6	; 0x8002d6 <_compareMatchHandler+0x6>
 814:	f0 91 d7 02 	lds	r31, 0x02D7	; 0x8002d7 <_compareMatchHandler+0x7>
 818:	30 97       	sbiw	r30, 0x00	; 0
 81a:	09 f0       	breq	.+2      	; 0x81e <__vector_8+0x30>
 81c:	09 95       	icall
 81e:	ff 91       	pop	r31
 820:	ef 91       	pop	r30
 822:	bf 91       	pop	r27
 824:	af 91       	pop	r26
 826:	9f 91       	pop	r25
 828:	8f 91       	pop	r24
 82a:	7f 91       	pop	r23
 82c:	6f 91       	pop	r22
 82e:	5f 91       	pop	r21
 830:	4f 91       	pop	r20
 832:	3f 91       	pop	r19
 834:	2f 91       	pop	r18
 836:	0f 90       	pop	r0
 838:	0f be       	out	0x3f, r0	; 63
 83a:	0f 90       	pop	r0
 83c:	1f 90       	pop	r1
 83e:	18 95       	reti

00000840 <__vector_13>:
 840:	1f 92       	push	r1
 842:	0f 92       	push	r0
 844:	0f b6       	in	r0, 0x3f	; 63
 846:	0f 92       	push	r0
 848:	11 24       	eor	r1, r1
 84a:	8f 93       	push	r24
 84c:	9f 93       	push	r25
 84e:	af 93       	push	r26
 850:	bf 93       	push	r27
 852:	80 91 16 02 	lds	r24, 0x0216	; 0x800216 <_timerUs>
 856:	90 91 17 02 	lds	r25, 0x0217	; 0x800217 <_timerUs+0x1>
 85a:	a0 91 18 02 	lds	r26, 0x0218	; 0x800218 <_timerUs+0x2>
 85e:	b0 91 19 02 	lds	r27, 0x0219	; 0x800219 <_timerUs+0x3>
 862:	81 50       	subi	r24, 0x01	; 1
 864:	90 48       	sbci	r25, 0x80	; 128
 866:	af 4f       	sbci	r26, 0xFF	; 255
 868:	bf 4f       	sbci	r27, 0xFF	; 255
 86a:	80 93 16 02 	sts	0x0216, r24	; 0x800216 <_timerUs>
 86e:	90 93 17 02 	sts	0x0217, r25	; 0x800217 <_timerUs+0x1>
 872:	a0 93 18 02 	sts	0x0218, r26	; 0x800218 <_timerUs+0x2>
 876:	b0 93 19 02 	sts	0x0219, r27	; 0x800219 <_timerUs+0x3>
 87a:	bf 91       	pop	r27
 87c:	af 91       	pop	r26
 87e:	9f 91       	pop	r25
 880:	8f 91       	pop	r24
 882:	0f 90       	pop	r0
 884:	0f be       	out	0x3f, r0	; 63
 886:	0f 90       	pop	r0
 888:	1f 90       	pop	r1
 88a:	18 95       	reti

0000088c <Usart_PutShort>:
 88c:	cf 93       	push	r28
 88e:	c8 2f       	mov	r28, r24
 890:	89 2f       	mov	r24, r25
 892:	0e 94 e8 00 	call	0x1d0	; 0x1d0 <Usart_PutChar>
 896:	8c 2f       	mov	r24, r28
 898:	0e 94 e8 00 	call	0x1d0	; 0x1d0 <Usart_PutChar>
 89c:	cf 91       	pop	r28
 89e:	08 95       	ret

000008a0 <DefaultMessageHandler>:
 8a0:	0f 93       	push	r16
 8a2:	1f 93       	push	r17
 8a4:	cf 93       	push	r28
 8a6:	df 93       	push	r29
 8a8:	ec 01       	movw	r28, r24
 8aa:	88 81       	ld	r24, Y
 8ac:	86 3a       	cpi	r24, 0xA6	; 166
 8ae:	39 f5       	brne	.+78     	; 0x8fe <DefaultMessageHandler+0x5e>
 8b0:	8c 81       	ldd	r24, Y+4	; 0x04
 8b2:	90 e0       	ldi	r25, 0x00	; 0
 8b4:	8c 01       	movw	r16, r24
 8b6:	16 6a       	ori	r17, 0xA6	; 166
 8b8:	0e 94 c3 00 	call	0x186	; 0x186 <EnterAtomic>
 8bc:	8c 81       	ldd	r24, Y+4	; 0x04
 8be:	81 30       	cpi	r24, 0x01	; 1
 8c0:	51 f4       	brne	.+20     	; 0x8d6 <DefaultMessageHandler+0x36>
 8c2:	ea 81       	ldd	r30, Y+2	; 0x02
 8c4:	fb 81       	ldd	r31, Y+3	; 0x03
 8c6:	c0 81       	ld	r28, Z
 8c8:	c8 01       	movw	r24, r16
 8ca:	0e 94 46 04 	call	0x88c	; 0x88c <Usart_PutShort>
 8ce:	8c 2f       	mov	r24, r28
 8d0:	0e 94 e8 00 	call	0x1d0	; 0x1d0 <Usart_PutChar>
 8d4:	11 c0       	rjmp	.+34     	; 0x8f8 <DefaultMessageHandler+0x58>
 8d6:	82 30       	cpi	r24, 0x02	; 2
 8d8:	59 f4       	brne	.+22     	; 0x8f0 <DefaultMessageHandler+0x50>
 8da:	ea 81       	ldd	r30, Y+2	; 0x02
 8dc:	fb 81       	ldd	r31, Y+3	; 0x03
 8de:	c0 81       	ld	r28, Z
 8e0:	d1 81       	ldd	r29, Z+1	; 0x01
 8e2:	c8 01       	movw	r24, r16
 8e4:	0e 94 46 04 	call	0x88c	; 0x88c <Usart_PutShort>
 8e8:	ce 01       	movw	r24, r28
 8ea:	0e 94 46 04 	call	0x88c	; 0x88c <Usart_PutShort>
 8ee:	04 c0       	rjmp	.+8      	; 0x8f8 <DefaultMessageHandler+0x58>
 8f0:	c8 01       	movw	r24, r16
 8f2:	99 27       	eor	r25, r25
 8f4:	0e 94 46 04 	call	0x88c	; 0x88c <Usart_PutShort>
 8f8:	0e 94 ca 00 	call	0x194	; 0x194 <LeaveAtomic>
 8fc:	1f c0       	rjmp	.+62     	; 0x93c <__stack+0x3d>
 8fe:	88 3a       	cpi	r24, 0xA8	; 168
 900:	e9 f4       	brne	.+58     	; 0x93c <__stack+0x3d>
 902:	0e 94 c3 00 	call	0x186	; 0x186 <EnterAtomic>
 906:	8c 81       	ldd	r24, Y+4	; 0x04
 908:	81 30       	cpi	r24, 0x01	; 1
 90a:	39 f4       	brne	.+14     	; 0x91a <__stack+0x1b>
 90c:	8d 81       	ldd	r24, Y+5	; 0x05
 90e:	ea 81       	ldd	r30, Y+2	; 0x02
 910:	fb 81       	ldd	r31, Y+3	; 0x03
 912:	80 83       	st	Z, r24
 914:	81 e0       	ldi	r24, 0x01	; 1
 916:	98 ea       	ldi	r25, 0xA8	; 168
 918:	0d c0       	rjmp	.+26     	; 0x934 <__stack+0x35>
 91a:	82 30       	cpi	r24, 0x02	; 2
 91c:	49 f4       	brne	.+18     	; 0x930 <__stack+0x31>
 91e:	8d 81       	ldd	r24, Y+5	; 0x05
 920:	9e 81       	ldd	r25, Y+6	; 0x06
 922:	ea 81       	ldd	r30, Y+2	; 0x02
 924:	fb 81       	ldd	r31, Y+3	; 0x03
 926:	91 83       	std	Z+1, r25	; 0x01
 928:	80 83       	st	Z, r24
 92a:	81 e0       	ldi	r24, 0x01	; 1
 92c:	98 ea       	ldi	r25, 0xA8	; 168
 92e:	02 c0       	rjmp	.+4      	; 0x934 <__stack+0x35>
 930:	80 e0       	ldi	r24, 0x00	; 0
 932:	98 ea       	ldi	r25, 0xA8	; 168
 934:	0e 94 46 04 	call	0x88c	; 0x88c <Usart_PutShort>
 938:	0e 94 ca 00 	call	0x194	; 0x194 <LeaveAtomic>
 93c:	df 91       	pop	r29
 93e:	cf 91       	pop	r28
 940:	1f 91       	pop	r17
 942:	0f 91       	pop	r16
 944:	08 95       	ret

00000946 <__udivmodsi4>:
 946:	a1 e2       	ldi	r26, 0x21	; 33
 948:	1a 2e       	mov	r1, r26
 94a:	aa 1b       	sub	r26, r26
 94c:	bb 1b       	sub	r27, r27
 94e:	fd 01       	movw	r30, r26
 950:	0d c0       	rjmp	.+26     	; 0x96c <__udivmodsi4_ep>

00000952 <__udivmodsi4_loop>:
 952:	aa 1f       	adc	r26, r26
 954:	bb 1f       	adc	r27, r27
 956:	ee 1f       	adc	r30, r30
 958:	ff 1f       	adc	r31, r31
 95a:	a2 17       	cp	r26, r18
 95c:	b3 07       	cpc	r27, r19
 95e:	e4 07       	cpc	r30, r20
 960:	f5 07       	cpc	r31, r21
 962:	20 f0       	brcs	.+8      	; 0x96c <__udivmodsi4_ep>
 964:	a2 1b       	sub	r26, r18
 966:	b3 0b       	sbc	r27, r19
 968:	e4 0b       	sbc	r30, r20
 96a:	f5 0b       	sbc	r31, r21

0000096c <__udivmodsi4_ep>:
 96c:	66 1f       	adc	r22, r22
 96e:	77 1f       	adc	r23, r23
 970:	88 1f       	adc	r24, r24
 972:	99 1f       	adc	r25, r25
 974:	1a 94       	dec	r1
 976:	69 f7       	brne	.-38     	; 0x952 <__udivmodsi4_loop>
 978:	60 95       	com	r22
 97a:	70 95       	com	r23
 97c:	80 95       	com	r24
 97e:	90 95       	com	r25
 980:	9b 01       	movw	r18, r22
 982:	ac 01       	movw	r20, r24
 984:	bd 01       	movw	r22, r26
 986:	cf 01       	movw	r24, r30
 988:	08 95       	ret

0000098a <memcpy>:
 98a:	fb 01       	movw	r30, r22
 98c:	dc 01       	movw	r26, r24
 98e:	02 c0       	rjmp	.+4      	; 0x994 <memcpy+0xa>
 990:	01 90       	ld	r0, Z+
 992:	0d 92       	st	X+, r0
 994:	41 50       	subi	r20, 0x01	; 1
 996:	50 40       	sbci	r21, 0x00	; 0
 998:	d8 f7       	brcc	.-10     	; 0x990 <memcpy+0x6>
 99a:	08 95       	ret

0000099c <_exit>:
 99c:	f8 94       	cli

0000099e <__stop_program>:
 99e:	ff cf       	rjmp	.-2      	; 0x99e <__stop_program>
